:100000008A110A1205280000090007309F00831694
:100010003C308500860183128601850106172F205A
:10002000061386162F20861286172F208613051793
:100030002F20051385172F20851305142F20051059
:10004000053084000230AA004130A0000330A10036
:100050005830A2000230A3008A200C282E28061651
:100060006430A000A1014F20061286156430A00064
:10007000A1014F20861106156430A000A1014F2078
:10008000061186146430A000A1014F2086100614CA
:100090006430A000A1014F20061008004E28A008DF
:1000A00003195A286120A00300000000000000008E
:1000B00000004F28A108031908006120A103A00334
:1000C0004F280C30A500A50B63280000000012305B
:1000D000A200A20B7028722072200000000008000D
:1000E000722069280D30A400A40B742800000800B9
:1000F0001030A8020001031C013EA902031C0800E5
:1001000081280A30A8020001031C013EA902031C39
:10011000080081282A0880042008A8002108A900D6
:1001200078200130A202031CA3032A0980052008BD
:10013000A8002108A9007820A208031D8A28A30886
:06014000031D8A280800DF
:02400E00503F21
:00000001FF
